:1000000015C01AC019C018C017C016C015C014C03A
:1000100013C012C011C010C00FC055C00DC00CC01D
:100020000BC03F065B4F666D7D077F6F11241FBEBF
:10003000CFEDCDBFE6D0B9C1E3CF0F931F93CF93E0
:10004000DF93262F803D37E0930710F08FEC97E089
:1000500031E0CAE0D0E001E010E0BE011AD1215049
:10006000422F437029F0FC01EE5DFF4FE49101C087
:10007000EAE0A22FB0E0A801022E01C0440F0A94CA
:10008000EAF78FEF840F8E23EE0F440F4195E423A0
:10009000A359BF4FE82BEC93315037FD02C0CB0181
:1000A000DCCF61157105D9F7822F837039F02150AB
:1000B000E22FF0E0E359FF4F1082F6CFDF91CF91AE
:1000C0001F910F9108951F920F920FB60F92112456
:1000D0002F933F934F935F936F937F938F939F9350
:1000E000AF93BF93EF93FF93389B36C0389824B1FA
:1000F00035B18091640090916500A0916600B09147
:100100006700820F931FA11DB11D8093640090931F
:100110006500A0936600B093670020916C002F5F8C
:1001200020936C002770E22FF0E081E090E001C0A6
:10013000880F2A95EAF7E359FF4F9081892B17BA68
:100140001ABA292F277028BB987F9BBB982F9770CE
:1001500097BB887F8ABB44C0389A24B135B180915F
:10016000680090916900A0916A00B0916B00820FC5
:10017000931FA11DB11D8093680090936900A09307
:100180006A00B0936B0020916C00211129C040914E
:100190006400509165006091660070916700452F82
:1001A000562F672F7727509361004093600010927D
:1001B0006400109265001092660010926700892F0B
:1001C0009A2FAB2FBB27909363008093620010920D
:1001D00068001092690010926A0010926B009F9A5A
:1001E000FF91EF91BF91AF919F918F917F916F910F
:1001F0005F914F913F912F910F900FBE0F901F90E5
:100200001895EDE6F0E081E098E09E0F282F20950C
:100210002193880F9E13FACF479A8EE080B98FEF13
:1002200081B988E685BF3F9A8CEF86B91C9A78948D
:1002300088959F9BFDCF609160007091610080E088
:1002400090E027EF30E040E050E039D05A0164E020
:10025000C5010396F2DE609162007091630080E058
:1002600090E02EE935E040E050E029D049015A0104
:100270004501AA24BB2481149104A104B10419F0FE
:10028000C401019702C080E090E068E0D6DE9F984C
:10029000CFCFAA1BBB1B51E107C0AA1FBB1FA617CC
:1002A000B70710F0A61BB70B881F991F5A95A9F71F
:1002B00080959095BC01CD01089568940010E89454
:1002C000A0E0B0E0E5E6F1E01DC0EFEFE7F959018D
:1002D0006A015E23550FEE08FE2C87019B01AC01DD
:1002E0009E23990F660B762FCB0131D0CDB7DD273A
:1002F000EAE01FC02F923F924F925F926F927F92DF
:100300008F929F92AF92BF92CF92DF92EF92FF9225
:100310000F931F93CF93DF93CDB7CA1BCDBFDD27BC
:1003200009942A88398848885F846E847D848C8407
:100330009B84AA84B984C884DF80EE80FD800C8110
:100340001B81AA81D981CE0FCDBFCA2F0895DF931B
:10035000CF939F92A0E49A2E0024D001E001F001F7
:1003600016950795F794E794D794C794B794A794F4
:1003700048F41068A20FB31FC41FD51FE61FF71F54
:10038000081E191E220F331F441F551F661F771F9B
:10039000881F991F9A9421F79D01AE01BF01C001EA
:0E03A00011249F90CF91DF910895F894FFCF24
:00000001FF
